:020000040000FA
:10000000F8020020DD000000E1000000E300000035
:1000100000000000000000000000000000000000E0
:10002000000000000000000000000000E5000000EB
:100030000000000000000000E7000000E9000000F0
:10004000EB000000EB000000510500006D05000012
:10005000EB000000EB000000EB000000EB000000F4
:10006000BD090000D9090000EB000000EB00000012
:10007000F5090000EB000000EB000000EB000000C1
:10008000EB000000EB000000EB000000EB000000C4
:10009000EB000000EB000000EB000000EB000000B4
:1000A000EB000000EB000000EB000000EB000000A4
:1000B000EB000000EB000000EB000000EB00000094
:1000C0000348854600F03CF8004800475D0F0000FB
:1000D000F8020020401EFDD2704700000348004790
:1000E000FEE7FEE7FEE7FEE7FEE7FEE7C1000000F1
:1000F00030B50B46014600202022012409E00D46C0
:10010000D5409D4205D31D469540491B2546954047
:1001100040191546521E002DF1DC30BD03460B433D
:100120009B0703D009E008C9121F08C0042AFAD2AD
:1001300003E00B780370401C491C521EF9D2704733
:10014000064C0125064E05E0E36807CC2B430C3C2A
:1001500098471034B442F7D3FFF7B6FF5C1C000099
:100160007C1C00000248016AC20111430162704711
:1001700000020050C10F8A00044951184A68C306A2
:10018000DB0E0120984002434A6070470002005095
:10019000F3B58BB00C46FFF7E5FF0B9800287448C9
:1001A000016813D0042211430160102000F0BCF953
:1001B0000120C00409906F480090042008906E4808
:1001C0006E49201888420ED800251DE08908890054
:1001D000491C0160012000F0A7F90020099068483F
:1001E00000900220EAE767486649201849428842A1
:1001F00002D80125640007E063486349201849429A
:1002000088427DD20325A4000026F643089F22E001
:1002100039460098FFF76CFF5C49844641185C48FA
:10022000814217D2554B02225B1C53486146514311
:10023000401C0818984209D8A14201D9081B00E0C7
:10024000601AB04202D2060004920CD05148521CEF
:100250008242EAD97F1C212FDAD900200696C043BA
:100260000190089E54E00999A803084301217A02ED
:100270008902511A08430499891E08433C490862BF
:10028000042000F051F9691C79430098FFF730FF12
:10029000049948430DB0F0BD31460098FFF728FFA0
:1002A0003A4942183A498A4231D20221324B024637
:1002B0004A435B1CD7185B429F4224D8A24201D913
:1002C000121B00E0A21A019B9A421CD20192069BCB
:1002D0000F469A4217D10999A803084301217202D7
:1002E0008902511A0843B91E0843214908620420B3
:1002F00000F01AF9691C71430098FFF7F9FE00E05D
:1003000008E07843C6E7234A491C9142CED9761CBF
:10031000212EC1D90B9800280FD01F491448016223
:10032000042000F001F91DA0006803901048016A44
:100330000013014203D00020ACE71949EEE708039F
:1003400001D50C4800E00E488A03A3D40A04920F9A
:1003500003AB9B5CCA058904D20DC90E891C8008B9
:10036000921C59435043FFF7C3FE800092E7000000
:100370000002005000805101FF1E0AFAFFE0F5055F
:10038000001BB700800F05FDC08782FEFF95E7FFC9
:10039000BF77CC00010200001844080001020204EB
:1003A00016400000044982070A6801D092089200B2
:1003B00002430A60704700000002005010B500F0D0
:1003C00059FA0148006810BD080000200448006880
:1003D0008007800F012801D0002070470148704736
:1003E00000020050001BB700044800688007800F1F
:1003F000022801D0002070470148704700020050D9
:10040000001BB70008B511A0006800901048016AF1
:100410000013014201D0002008BD080301D50D489A
:1004200000E00D488A03F7D40A04920F6B469B5CE8
:10043000CA058904D20DC90E891C8008921C594333
:100440005043FFF755FE800008BD00000102020482
:100450000002005000805101001BB70008B511A038
:10046000006800901048016A0013014201D000208A
:1004700008BD080301D50D4800E00D488A03F7D4F4
:100480000A04920F6B469B5CCA058904D20DC90E03
:10049000891C8008921C59435043FFF729FE8000B5
:1004A00008BD00000102020400020050008051015A
:1004B000001BB70010B5074A93691B091B010B43CA
:1004C00093611169C908C9000143116100F0D2F9B3
:1004D00010BD00000002005070B5430E1B070DD088
:1004E00043009B0F0F4C9B001C192368C5002D0F68
:1004F000C601F60EB540AB430B432360840A2106C8
:10050000090E0DD00103074B890F89000833CB1862
:1005100019688005E4B2C00E8440A14311431960FC
:1005200070BD00001002005010B50749074A05E0F1
:100530000B46491E002B01DC002010BDD468034689
:10054000A343F5D1012010BD80F52000000200502A
:1005500004490420086204484068002800D000478D
:1005600070470000C04000502000002004490420D3
:10057000086204480068002800D000477047000067
:10058000404100502000002010B5094A002305E03A
:100590001178521C0029FBD15B1CDBB2834202D0D4
:1005A00011780029F4D1014602A001F075F810BDC0
:1005B000881B00004572726F723D257520257300FF
:1005C000F0B500230125944603272A469A400A42A3
:1005D00009D006685C003A46A2409643224664462B
:1005E0009440264306605B1C082BEED3F0BD000050
:1005F0008307FF22DB0E9A408907090E99400028E5
:100600000BDA0007000F0838830808489B00181809
:10061000C36993430B43C3617047830804489B003D
:100620001B181868904308431860704700ED00E0FD
:1006300000E400E0FFB581B004461D4600261946DF
:10064000039800F090FA694608702946039800F074
:1006500097FA47190121684600F092FA3818029972
:10066000C01C88422FD8C02601220021DC2326701E
:10067000DB2014E0039F7F5CC02F02D0DB2F09D169
:1006800004E0A054521CD2B2A35404E0A054521C63
:10069000D2B2DD27A754521C491CD2B2C9B2A9421A
:1006A000E8D30021DD256F467F5CC02F0ED0DB2F05
:1006B00011D0A754521C491C0906D2B2090EF2D01F
:1006C000A654521CD6B2304605B0F0BDA054521C00
:1006D000D2B2A354EEE7A054521CD2B2A554E9E71B
:1006E0008168082291438160704710B5029C202BDD
:1006F00000D10023DB000B4313430360012292046B
:10070000914201D110218160214600F001F810BD15
:1007100070B5064619480D4641698906890F21D0F2
:1007200040698006800F022823D0FFF747FE044669
:10073000A54200D90546002D1ED029462046FFF7C8
:10074000D7FC401C4008401EFF2800D9FF207168DC
:10075000090A09020143716041002046891CFFF724
:10076000C7FC70BDFFF732FE0400E1D1FFF73CFE8D
:10077000DDE7FFF773FEDAE7002070BD00020050EE
:10078000F8B55921304C1622882021602260206063
:100790002368002BF9D02D4D04202860FFF702FEBE
:1007A0000820FFF7FFFD1020FFF7BEFE2869072194
:1007B00008432861A86900090001A8612449A8022A
:1007C000FFF7E6FC01210220FFF774FE2148FFF746
:1007D000D1FC214E3046FFF7CDFCB3221204082194
:1007E0003046FFF779FE1D48FFF7C4FC1C48FFF7B1
:1007F000C1FC00F03FF81BA000680090286A291394
:1008000001400025002901D02A4616E0010301D548
:10081000154A00E0154A81030FD40104890F6B4685
:100820005E5CC3058004C10EDB0D891C90089B1C17
:1008300071435843FFF75CFC82000D4E7260FFF776
:10084000BDFDB0602560F8BD000100500002005001
:1008500000E1F505103D80A71CFE23A61400C0A7EB
:100860001500E0A70102020400805101001BB7003F
:1008700010000020F8B520A00068204E0090316ADA
:1008800030131F4C1F4F014201D0002016E0080317
:1008900001D5204600E038468A030FD40A04920F9F
:1008A0006B469B5CCA058904D20DC90E891C800861
:1008B000921C59435043FFF71BFC8000124D2860E7
:1008C00031694907490F12D0022902D0032910D0FB
:1008D0002046B1690907090F491CFFF709FC0B49BC
:1008E00068604A108018FFF703FCA860F8BD38461E
:1008F000EFE70748EDE700000102020400020050A4
:1009000000805101001BB7000400002040420F008E
:10091000102700000F4A10499042486901D1000A8F
:1009200000E0000B4007400F06D001280ED002283F
:100930000ED00A480068704708688007800F0128B9
:1009400002D00120C0037047054870470548704732
:100950000548EFE7000001400002005000000020C1
:10096000001BB7001027000008000020F8B5134650
:100970000F460646FFF7CEFF044600254008984282
:1009800001D2022010E0012149068C4202D3032546
:10099000A40805E0012109068C4201D30125044683
:1009A00019462046FFF7A4FB2F43376070606D1C8B
:1009B000684301462046FFF79BFBF8BD0449012030
:1009C000886004480068002800D000477047000095
:1009D00000000140280000200449012088600448EC
:1009E0004068002800D00047704700002000014008
:1009F0002800002010B51849C869C207174812D04E
:100A00000A68D3B24289202A0DDA521C4281028937
:100A1000841820342373521CD317DB0E9B185B09F8
:100A20005B01D21A0281CA6992070FD58288521ED1
:100A30000DD38280028883181B7B0B60521CD11758
:100A4000C90E891849094901511A018010BD486829
:100A500002229043486010BD00000540980000202D
:100A600070B51B4E0D4604467169002089010322B2
:100A7000890F2063E260A06000291FD001291FD0E8
:100A8000022901D313480068B1690905090F491CFF
:100A9000FFF72EFB0646002D19D06808801929465D
:100AA000FFF726FB0C49801E88420CD9E80080190C
:100AB0002946FFF71DFB0009801E07E00748E3E712
:100AC000FFF7A0FCE0E7032109070843606270BD5F
:100AD0000002005000000020FFFF0000001BB700D4
:100AE00010B518480178401C3F290ED0532901D079
:100AF00073290DD100783038030000F027F80A0A76
:100B00000C10121416181A1C1E200F4800F026FE96
:100B100010BD002000E00120FFF736FD10BD0220CF
:100B2000FAE70320F8E70420F6E70520F4E70620BB
:100B3000F2E70720F0E70820EEE70920ECE70A20BB
:100B4000EAE70000E4000020BC1A000030B474465C
:100B5000641E2578641CAB4200D21D46635D5B00B9
:100B6000E31830BC1847034610B50020024604E0E5
:100B70009C5C2018521CC0B2D2B28A42F8D310BD7D
:100B8000034610B50020024608E09C5CC02C01D052
:100B9000DB2C01D1401CC0B2521CD2B28A42F4D329
:100BA00010BD00001FB507206A461070002151706B
:100BB00051800A4991804900D180107203205072FF
:100BC000074850817D20400190818810D0811021FC
:100BD000104600F019F904B010BD00001027000005
:100BE000B80B000002E008C8121F08C1002AFAD1A1
:100BF00070477047002001E001C1121F002AFBD19D
:100C0000704710B504460089FFF764FA6168012057
:100C100008606089FFF75EFA61680020086020893B
:100C2000FFF758FA10BD70B504460068012505604D
:100C30002089FFF74FFA606805602089FFF74AFABC
:100C4000206800686168C5B2002008602089FFF74D
:100C500041FA284670BDF8B50026044635463746A9
:100C600076002089FFF736FA616801200860208944
:100C7000FFF730FA206800683043C6B2606807604A
:100C80002089FFF727FA6D1CEDB2082DE8D3304616
:100C9000F8BD70B5044621680120086061680860ED
:100CA0002089FFF717FA2068002505602089FFF7E3
:100CB00011FA606805602089FFF70CFA70BD70B505
:100CC00004462168002008606068012505602089CD
:100CD000FFF700FA2068056070BD70B506460D4646
:100CE00000243168E80908603046FFF78AFF68068B
:100CF000641C050EE4B2082CF3D370BD0A48016AE7
:100D000001221143016205200007416B074A11408F
:100D10004163416B08221143416305484168120455
:100D2000114341607047000000000E40F7F7FFF7E5
:100D3000404000500B4908224A620A4A40329368F8
:100D40001B091B019B1D93600A6A0123DB021A43E6
:100D50000A620A6B1207FCD409688905890D0180B3
:100D60007047000000000E400949C20704D08A699C
:100D7000002A09D000228A61800704D5486A002829
:100D800004D00020486270470122F4E70120F9E70F
:100D90004042005010B505200007816B8163C16B94
:100DA000C163012240210748FFF70AFC05480122E0
:100DB00002214030FFF704FC0348002181614162B9
:100DC00010BD000080400050404200507CB50C49EE
:100DD0000C4C03C90191009021786D468900695837
:100DE000FF200026002908D088472178491CC9B275
:100DF000217089006958002900D126707CBD00004F
:100E0000B41A00003000002030B591B00D460B46FA
:100E10000246202108A8FFF70DFC0446202D33D2FE
:100E20008E21202000F08AF80021FD2000F086F8B5
:100E3000F020FFF74FF968460470224608A9401CCD
:100E4000FFF76CF96D4620240021FD2000F076F8B4
:100E50004B200001FFF73EF922462946A02000F072
:100E600057F80A48816A0029FCD17021272000F038
:100E700065F80021E12000F061F80021FD2000F07C
:100E80005DF8304611B030BDFF20FBE780420050D6
:100E90001CB503200521084C024601910090042353
:100EA0002146064800F000FA0449224608460C3064
:100EB00000F0F2F91CBD00000300030080000020D8
:100EC000F8B50E460093C1B21346069D079C324604
:100ED000064800F019FA002803D0002D00D0A847DA
:100EE000F8BD002CFCD0A047F8BD00008000002019
:100EF0000649086208680122104308600868C04378
:100F0000C007FBD00869C0B2704700000000034072
:100F1000F8B50F46084E002115467160FFF7E8FF4F
:100F2000002404E0385DFFF7E3FF641CE4B2AC4248
:100F3000F8D301207060F8BD0042005070B50D4636
:100F4000054C00216160FFF7D3FF2846FFF7D0FF73
:100F50000120606070BD000000420050FFF710FCEF
:100F6000FFF796FF00F038F9012000F057F8FFF77F
:100F7000C5FE00F01DF9FF201849F53000F012FA07
:100F8000E120400200F092FB154800F0E7FB15A0BD
:100F900000F0E4FB0222012119A000F07DFB00F02B
:100FA000F5F8FFF7F7FE1A4D7C260320FFF7DCFE6D
:100FB0001848FFF7BFFE34462846FFF78BF8641E3B
:100FC000FAD2FFF703FF3E2000F0B0FB10211248D9
:100FD00000F058FAFFF784FDE7E700007512000003
:100FE0000E1900003232382D3730343520466978FA
:100FF00074757265206D6F6E69746F720000000009
:101000002C5665722025752E253032750A00000099
:10101000086100001C000020E4000020F8B5044630
:101020005920524D1622882128602A6029602B6899
:10103000002BF9D04E48FFF79DF84E48FFF79AF87D
:10104000FFF718FC00232B6005221207906B4A491A
:1010500008409063916B01208002014391634749EE
:101060008D68092635438D60956B454E35409563F7
:10107000956B4600354395638D68902635438D60AA
:10108000956B404E35409563956B8600354395636F
:101090008D680926360235438D60956B3A4E354092
:1010A0009563956BC600354395638A6809252D03C2
:1010B0002A438A600D68FF221202954326023543B7
:1010C0000D604D6807273F02BD43281848608868B7
:1010D000400040088860CB627D20C00048610D68F8
:1010E0002D0A2D0225430D604D687027BD43403504
:1010F0004D608D686D006D088D608B6208610D68B4
:101100002D0A2D0225430D604C68E408E400241DDF
:101110004C608C68640064088C604B62C8600C682A
:10112000944334430C604A683C02A2430124A40364
:1011300012194A608A68520052088A600B638861FB
:1011400088680122104388608868102210438860F4
:1011500088688A1510438860886812011043886087
:101160004B628B62CB620B63F8BD00000001005044
:101170001400C0A71500E0A7FBFBFFFF0000044020
:10118000F7F7FFFFEFEFFFFFDFDFFFFF1CB507A063
:10119000006801906720009020230222032101A80B
:1011A00000F0ACF900F044FA1CBD0000A55A110093
:1011B0001CB508A00068019000F00EF82C200090EB
:1011C0000D231422032101A800F098F900F026FA5B
:1011D0001CBD000023232300F8B505242407206B41
:1011E0002063206B07256D03284320631348416863
:1011F0004160134E3046FEF7BDFF012210213046FC
:10120000FFF76AF9012202210E48FFF7D9F90022FF
:1012100004210D48FFF7D4F9206B284320630B48C5
:101220000B4C00900823042200212046FFF75DFAB2
:101230002046FFF755FA00202062F8BD400000501C
:101240000C0040A6004000504041005080841E0029
:101250000000034006490862086801221043086044
:101260000868C043C007FBD00869C0B270470000DF
:10127000000003401CB506490220088000200090B1
:1012800001901223034A10217620FFF719FE1CBD9E
:10129000100000204000002010B51AC91AC00C38F8
:1012A000511C00D0826010BDF8B58C460546500137
:1012B000990041181348069F0918079E29607C0170
:1012C000B100611808186860012460462146994001
:1012D000A8609001A2031043052212078018022281
:1012E000FFF76EF9B4400122B801920310430522C2
:1012F0001207801821460222FFF762F92846FFF7FD
:10130000DEFCF8BD00420050FFB581B01F460E461E
:101310000546002472B6FFF7BCFC7600F1B2284601
:10132000FFF7DBFC2846FFF77EFC002832D1284679
:101330000399FFF7D2FC2846FFF775FC002829D156
:101340002846FFF7A6FC761CF1B22846FFF7C5FC3D
:101350002846FFF768FC00281CD10A9E761E0CE088
:10136000FFF779FC38552968002008602846FFF708
:1013700048FC296801200860641CB4422846EFD369
:10138000FFF769FC38552968012008602846641C6D
:10139000FFF737FC2846FFF792FC62B6204605B0FF
:1013A000F0BD000070B504460D460F48FEF7E2FEA2
:1013B00022460E4C0121C9062046FFF7D7FA002D20
:1013C0000AD0206861030843206048150849086076
:1013D00002210820FFF70CF906480560206801216A
:1013E00089070843206070BD020080AE0000014004
:1013F00000E100E0280000200D4A50890028FCD0C0
:10140000D18850182030007B491CCB17DB0E5B18AD
:101410005B095B01C91AD180012306491B030B60DC
:101420005189491E5181034980390B607047000082
:101430009800002080E100E00F4A91882029FCD22A
:10144000518853181873491CC817C00E401840091A
:101450004001081A50800120084900030860918863
:10146000491C918006494A6802231A434A6003498D
:1014700080390860704700009800002080E100E09B
:1014800000000540F8B5144E0746B068002821D08A
:1014900000244D1EB068804700281BD00D2810D0B6
:1014A000082809D02028F5DBAC42F3DAC0B2385561
:1014B000641C00F03BF9EDE7002CEBD00820641E23
:1014C000F7E7002038550D2000F030F90A2000F031
:1014D0002DF90120F8BD00003400002010B50021D6
:1014E000E12000F0C9F80021E22000F0C5F810BDAD
:1014F00010B57021272000F0BFF810BDFFB50D46D4
:101500003EA003C887B0019100903EA000683EA1B4
:10151000049003C9039102903DA0006805903DA08E
:10152000006806901E465A21532000F0A5F8A52118
:10153000532000F0A1F80124374F02E03846FEF7AF
:10154000C9FD641EFAD2FFF7C9FFFFF7D1FF212EB4
:1015500001D2002100E018213D2000F08DF800218B
:10156000FD2000F089F80321222000F085F8A81E54
:10157000C1B2232000F080F82520099900F07CF802
:101580003146312000F078F83146322000F074F80E
:101590002A463020079900F059F82A462A20079950
:1015A00000F054F8052269463F2000F04FF806226B
:1015B00002A93A2000F04AF8012205A9392000F0DA
:1015C00045F8032204A93E2000F040F8032206A9B2
:1015D0003B2000F03BF800213C2000F04DF8262095
:1015E000109900F049F80021242000F045F800216E
:1015F000212000F041F80BB0F0BD000012ED679C17
:1016000046000000F63F5D004521EF2C5A400000E7
:10161000010000000BDF02000861000010B58F21FF
:10162000202000F029F80021FD2000F025F810BD51
:1016300010B58E21202000F01FF80021FD2000F0C1
:101640001BF8F020FEF746FD10BD0000F8B50F4670
:10165000084E002115467160FFF7FCFD002404E0F0
:10166000385DFFF7F7FD641CE4B2AC42F8D301200B
:101670007060F8BD0042005070B50D46054C002169
:101680006160FFF7E7FD2846FFF7E4FD0120606099
:1016900070BD0000004200500FB410B503A90298BD
:1016A00000F066F810BC08BC04B0184710B504463A
:1016B0001348FEF75FFD144912484860134841681B
:1016C00001225204914341602146114C2046FFF70C
:1016D000C7F9606811210843606001200D490003CB
:1016E00008600D490020088048808880C8800881F3
:1016F00048810B49094808600B490A48086010BD39
:10170000103D80A7030300004000005040410050FE
:101710000000054000E100E09800002039140000BE
:1017200034000020F91300003C00002010B50446EE
:101730000A2802D10D20FFF7F9FF07494A68002A5D
:1017400003D01470521C4A6010BD09680029FBD0F8
:101750002046884710BD00003400002010B5044624
:1017600002E0641CFFF7E2FF20780028F9D110BDE9
:10177000F3B58BB006463078761C002877D0252844
:1017800002D0FFF7D3FFF6E7002002903478761CF2
:10179000302C02D02D2C02D005E0012000E00220E8
:1017A00002903478761C002705E00A2047433F1951
:1017B0003478761C303F204630380928F5D96C2C17
:1017C00001D04C2C05D102980421084302903478B2
:1017D000761C002C4BD02146612C01D32039C9B294
:1017E0004F2937D006DC422932D043292AD0442958
:1017F00006D13DE0532905D0552939D0582939D093
:101800002046BEE70C98002420C80C9000E0641C21
:10181000285D0028FBD102E02020FFF787FF029817
:10182000800703D42046641CB842F5D32846FFF74E
:1018300095FF02E02020FFF779FF2046641CB842A4
:1018400099D2F7E70C980178001D0C90084698E7AC
:10185000022000E0082001900298400701D44429AA
:101860000AD00C9A442901CA0C9208D00EE04CE030
:101870000A20F0E71020EEE70C9901C90C9100282E
:1018800004DA02994042082211430291002501998D
:10189000FEF72EFCC9B2092904D9782C16D00722EC
:1018A0005118C9B204AA303151556D1C002801D01D
:1018B000102DECD30298000702D52D2151556D1C37
:1018C00002982C46C00703D0302002E02722E7E729
:1018D0002020089002E00898FFF728FF0298800770
:1018E00003D42046641CB842F5D304A86D1E405DA5
:1018F000FFF71CFF002DF8D102E02020FFF716FFB4
:101900002046641CB8429BD2F7E70DB0F0BD2A2AEE
:101910002A2A2A2A2A2A2A2A2A2A2A2A2A2A2A2A27
:101920002A2A2A2A2A2A2A2A2A2A2A2A2A2A2A2A17
:101930002A2A2A2A2A2A2A2A2A2A2A2A2A0A20203B
:101940002323232023232323232323202323232070
:101950002020202320202020202320232323232372
:1019600023232023202020202023200A202020237E
:101970002020232020202020202020232020202061
:10198000202320202020202320232020202020204E
:101990002020232020202320200A20202023202054
:1019A000232020202020202020232020202020232E
:1019B0002020202020232023202020202020202021
:1019C000202320232020200A20202023202023231E
:1019D00023232320202020232020202020232020F8
:1019E00020202023202323232323202020202020E5
:1019F00023202020200A20202023202023202020F4
:101A000020202020202320202020202023202020D0
:101A100023202023202020202020202020232023BA
:101A20002020200A202020232020232020202020C6
:101A3000202020232020202020202023202320209D
:101A4000202320202020202020202320202023208D
:101A5000200A202023232320232020202020202090
:101A60002323232020202020202023202020202367
:101A70002323232323232023202020202023200A64
:101A80002A2A2A2A2A2A2A2A2A2A2A2A2A2A2A2AB6
:101A90002A2A2A2A2A2A2A2A2A2A2A2A2A2A2A2AA6
:101AA0002A2A2A2A2A2A2A2A2A2A2A2A2A2A2A0AB6
:101AB00000000000A50B0000000000005330202DA6
:101AC000205265496E697420746F20746573740ABE
:101AD0005331202D20546573742073746570206F0A
:101AE0006E650A5332202D2054657374207374651B
:101AF000702074776F0A5333202D2054657374203F
:101B0000737465702074687265650A5334202D20E3
:101B100054657374207374657020666F75720A5310
:101B200035202D20546573742073746570206669A8
:101B300076650A5336202D205465737420737465BE
:101B400070207369780A5337202D205465737420F0
:101B50007374657020736576656E0A5338202D2086
:101B60005465737420737465702065696768740ABE
:101B70005339202D20546573742073746570206E62
:101B8000696E650A000000004F4B004144305F451C
:101B90005252004144310041443200414433004E2E
:101BA0004F5F5041544800494E56414C49445F4EA6
:101BB000414D450044454E4945440045584953541C
:101BC00000494E56414C49445F4F424A45435400F8
:101BD00057524954455F50524F5445435445440071
:101BE000494E56414C49445F4452495645004E4F78
:101BF000545F454E41424C4544004E4F5F46494C70
:101C0000455F53595354454D004D4B46535F414238
:101C10004F525445440054494D454F5554004C4F84
:101C2000434B4544004E4F545F454E4F5547485F28
:101C3000434F524500544F4F5F4D414E595F4F50F7
:101C4000454E5F46494C455300494E56414C494428
:101C50005F504152414D4554455200007C1C0000EC
:101C60000000002040000000E40B0000BC1C00004D
:101C700040000020B8020000F40B00000080510179
:101C80000080510100000000000000000000000082
:101C90000000000000000000000000000000000044
:101CA0000000000000000000000000000000000034
:0C1CB00000000000000000000000000028
:04000005000000DD1A
:00000001FF
